:020000040000FA
:100000006307300A070C02004000050006000700E5
:100010000A0AFF0C0D09220000000E080B0C240038
:10002000150C2A00AA0C2000A402EA02130A0B0CE9
:100030002400EB0C2A006002A402EA031B0A6A00F7
:10004000EA00CA01AA006A032A03690C2A00AA036B
:100050002A016A01AA016A02960D690E690F400A17
:1000600004006306340A330A100C24006000030500
:100070002304430403020003400320002100000A7C
:10008000EC000C0225004509400A0000EE0C2A0095
:10009000010C2B00EA024A0A0400EB024A0A00089B
:020FFE00000AE7
:00000001FF
